:020000040000FA
:02000000622874
:0800080085150B118B10A200FD
:10001000030EA3008312A300861C1B28061D25289F
:10002000861D2F28061E3A28861E4428061F4D28A6
:10003000861F57280C28A930A5000C30A400A50B5A
:100040001F28A40B1F2800005C282330A5000230C5
:10005000A400A50B2928A40B292800005C28F63051
:1000600081002230A5000230A400A50B3528A40B86
:1000700035285C28F530A5000330A400A50B3E28E8
:10008000A40B3E2800005C285B30A5000330A400D0
:10009000A50B4828A40B48285C28E030A5000230B6
:1000A000A400A50B5128A40B512800005C28BB30EC
:1000B000A500A50B59280000230E8300A20E220ED6
:1000C000851109008601850107309F008316FF30E6
:1000D00086003030850081138312861C7D28061D22
:1000E0008028861D8328061E8A28861E9128061FC2
:1000F0009828861F9F286D286D2890308B00A72890
:1001000090308B00A7288316283081008312A030FE
:100110008B00A7288316283081008312A0308B0023
:10012000A7288316623081008312A0308B00A72895
:100130008316653081008312A0308B00A7288316B8
:10014000673081008312A0308B00A72806140608B0
:10015000A60026100608A700271026082702031964
:04016000AA286D2834
:02400E00613F10
:00000001FF
